:020000040000FA
:040008005C2D080063
:100020008A150A1601208A110A122726F012F212E6
:10003000F2137113F113C001C1018B1786117011F6
:1000400083120313F801F901FA01FB01FC01FD0120
:10005000FE01FF01203084006F25A0002430200223
:100060000319FD283C302002031D2C28840AC901F5
:100070000230BD006F25C907D6208000840ABD0B61
:100080003A282208C800210EC80406304802BD00E4
:100090006F25C907D6208000840ABD0B482802308E
:1000A000BD006F25D6208000840ABD0B51286F2526
:1000B000BC003E303C02031D842884030008BC00C1
:1000C0008403000EBC0449083C02031D8D288313E1
:1000D000243084000008CA008403000ECA04CA0841
:1000E000031981284E304A0203188128061186150B
:1000F00090304A0707300318013E8A004A089027CB
:100100001E280030BF009C280130BF009C28023010
:10011000BF009C280330BF009C280430BF009C28EF
:100120000530BF009C280630BF009C280730BF0068
:100130009C280830BF009C280A30C8000030CA0044
:100140008317103084003F08800006157015BE2507
:100150001E2841346C346C34203459346F34753477
:100160007234203442346134733465342034413481
:10017000723465342034423465346C346F346E34F8
:0E0180006734203454346F34203455347334D3
:10019000F6308100D428EC308100D428D83081009A
:1001A000D4283D308100D4280B110800F700F60058
:1001B0000F30F605473077020318E4284130770204
:1001C000031CE4280930F60776080800B800B900D7
:1001D000F030B905390EF220B9000F303805F220A1
:1001E000B8000800F6000A307602031CFA283730FF
:1001F0007607FC283030760708000530BD00213036
:1002000084006F258000840ABD0B0129BC000D30DD
:100210003C02031D812830306C2532306C251E28AD
:100220000E30C8000130CA008A110A165A218A11FC
:100230000A127015BE2508001230C8000230CA002C
:1002400038267015BE2508000E30C8000430CA00DC
:1002500070150230D5008A150A1608208A110A1274
:10026000711C35290730BF00D9247015BE25080040
:100270000830C8000530CA0083132608BC00250ECC
:10028000BC04BC080319452947294E27482947279C
:10029000BE2508000830C8000630CA002608C20083
:1002A000250EC2042808C300270EC3042908C40071
:1002B0002A0EC404BE2508000A30C8000730CA0050
:1002C0008A110A1666218A110A127015BE250800C5
:1002D0000A30C8000830CA009F267015BE250800E5
:1002E0000830C8000930CA002608C100250EC10424
:1002F000BE2508000830C8000A30CA002608BC0025
:10030000250EBC04F212BC0803198729F216BE257B
:1003100008000830C8000B30CA002608BC00250EB3
:10032000BC04BC08031995299C298A110A160D26BC
:100330008A110A12F213A2298A110A160D268A11AD
:100340000A12F217BE2508000830C8000C30CA0097
:100350002608BC00250EBC047213BC08031DB1297D
:1003600072170B30D5008A150A1608208A110A1256
:10037000BE2508000800080083120313F0160610BB
:1003800008000830C8001230CA00BE250800083036
:10039000C8001B30CA008A110A16DC248A110A120E
:1003A0000430D500862408000830C8001E30CA007A
:1003B0008A110A16DC248A110A120330D50063243C
:1003C00008000830C8002330CA008A110A16E22447
:1003D0008A110A121C30D500632408000830C800B6
:1003E0002430CA008A110A16E2248A110A121D302A
:1003F000D500862408000830C8002530CA00BE2574
:100400008A110A1643218A110A1208000830C8000E
:100410002630CA008A110A1639218A110A12BE250D
:1004200008000830C8002730CA008A110A162521A2
:100430008A110A12BE2508000830C8002830CA00F8
:100440008A110A1624218A110A12BE25552C083059
:10045000C8002930CA008A110A1609208A110A1216
:10046000BE2508000830C8002A30CA0083132608B9
:10047000BE00250EBE048A110A1601268A110A1230
:10048000BE2508000830C8002B30CA002608BC0072
:10049000250EBC0400303C020319592A01303C02ED
:1004A00003196D2A02303C020319572A802A0D27AE
:1004B000802A0D275825FA2658253F278719802A94
:1004C0003727871587113F27D1208719802A0B1DD1
:1004D000652A0730BF00D924802A0D275825FA261F
:1004E0003727871587113F271930D5008A150A1637
:1004F00008208A110A12711C802A0730BF00D924F3
:10050000BE2508000A30C8002C30CA00F218902A14
:1005100072198E2A0030CA0003309E2A02309E2AA9
:100520003F27871D9C2A5030BD00871D9C2ABD0394
:10053000031D952A00309E2A01309E2ABC00831795
:1005400010308400831203133C0880007015BE2510
:1005500008000D275825FA260830C8002D30CA009B
:10056000BE2508000830C8002E30CA008711372782
:1005700087112E27071EC22A8A150A1671228A1190
:100580000A12B92A87155425542587113F27BE25FD
:1005900008000830C8002F30CA001A30D500442D9A
:1005A0000830C8003030CA001930D500442D08305A
:1005B000C8003130CA00E5248A110A160D268A11B6
:1005C0000A12EC2408000830C8003230CA000125A5
:1005D0008A110A160D268A110A120D250800083004
:1005E000C8003330CA002608BC00250EBC04003009
:1005F0003C02031DFD2A0D270C2B01303C02031D7C
:10060000032BFA260C2B02303C02031D092BE72694
:100610000C2B0630BF00D924BE2508000A30C800C4
:100620003430CA00831710308400AA2683120313C3
:100630001E08831203178000831203137015BE2552
:1006400008000A30C8003530CA0083171030840013
:10065000E726A6260D27831203131E08831203170D
:100660008000831203137015BE2508000A30C800ED
:100670003730CA008A110A1601268A110A12831716
:1006800010308400AE26831203131E088312031752
:100690008000831203137015BE2508000830C800BF
:1006A0003930CA0001258A150A16EC208A110A126F
:1006B000F11C5D2B70160730BF000D2508000830B7
:1006C000C8003B30CA002508BC0001303C020319B9
:1006D0006D2B0630BF00D924772B8A110A16E5242A
:1006E0008A110A12711D772B0730BF00D924BE254D
:1006F00008000830C8003C30CA00F801F901FA01CE
:10070000FB01FC01FD01FE01FF018A150A16EC2028
:100710008A110A123F27871D8A2B912B0730BF00B1
:10072000D924BE2508001030C8003D30CA0070151D
:100730000D30D500442D0830C8003E30CA00E524F5
:100740008A110A16E2228A110A12EC248A110A126C
:1007500008000830C8003F30CA0001258A110A1677
:100760001F238A110A120D2508000830C8004030E6
:10077000CA00E5248A110A16E2228A110A12EC2420
:1007800008000830C8004130CA0001258A110A1645
:100790001F228A110A120D2508000830C8004230B5
:1007A000CA00B7248A110A1600208A110A12BE252F
:1007B00008000830C8004330CA0001258A110A1613
:1007C0001F228A110A120D2508000830C800443083
:1007D000CA0001258A110A169C218A110A120D25C8
:1007E00008000830C8004530CA0001258A110A16E1
:1007F0006C218A110A120D2508000830C800463005
:10080000CA0001258A110A161F228A110A120D2513
:1008100008000830C8004730CA00E5248A110A16CB
:10082000E2228A110A12EC248A110A120800083006
:10083000C8004830CA00E5248A110A16AE228A117F
:100840000A12EC2408000830C8004930CA00E52428
:100850008A110A168D228A110A12EC240800083027
:10086000C8004A30CA00E5248A110A16E2228A1119
:100870000A12EC2408000830C8004B30CA002608D1
:10088000C000250EC004BE2508000830C8004C304A
:10089000CA00BE2558250F2608000830C8004D3074
:1008A000CA00BE2558251B2608000030BF000A30AC
:1008B000C8000030CA008317103084003F08800051
:1008C0007015BE250800B7248A150A1608208A115B
:1008D0000A12711C6F2C0730BF00D924842CBE254E
:1008E00050257B306C255025C9018A150A16B82180
:1008F0008A110A124908E62039086C2538086C2547
:1009000050257D306C255025BE250800B7248A155A
:100910000A1608208A110A12711C922C0730BF0097
:10092000D924B52CBE256F257B3C03199B2C0130A7
:10093000BF00D924B52CC9018A150A16CF218A1106
:100940000A126F25D620BC00BC0E6F25D6203C04B1
:1009500049020319AE2C0430BF0070166F257D3C90
:100960000319B52C0130BF00D924BE25080083131C
:100970002C08F8002B0EF8042A08F900290EF904B7
:100980002808FA00270EFA042608FB00250EFB04AF
:100990003408FC00330EFC043208FD00310EFD0467
:1009A0003008FE002F0EFE042E08FF002D0EFF045F
:1009B00008000A30C8000030CA00701583171030D4
:1009C00084003F08800006150800B724BE25502586
:1009D0007B306C25C90108004908E62039086C25E0
:1009E00038086C257D306C25FF2C0A30C80000309B
:1009F000CA0070158317103084003F088000BE25A0
:100A000008007012B724BE256F257B3C03190B2DFF
:100A10000130BF007016C90108006F25D620BC0048
:100A2000BC0E6F25D6203C04490203191A2D043050
:100A3000BF0070166F257D3C0319212D0130BF00CA
:100A4000701603138312701E2F2D0A30C800003059
:100A5000CA0070158317103084003F088000BE253F
:100A60000800E6203908C9076C253808C9076C2535
:100A700008006F25C907D620B900B90E6F25C90730
:100A8000D620B904390808008A150A1608208A11E8
:100A90000A12711C4E2D0730BF00D924BE25080054
:100AA000C8200B1D512D0800CE200B1D552D080010
:100AB000D1200B1D592D0800F300030E8301F50012
:100AC0000A08F4008A010B18002074088A00750EC9
:100AD0008300F30E730E0900F01C802DA52DF01C71
:100AE000722D8E2D83120313F01A7E2D0614831699
:100AF000891B7B2D782D831206100808061008002C
:100B0000F01A8D2D83128C13880006148316091B8E
:100B1000872D83128C1F8A2D061008008312031361
:100B20008C1A962D86128C1A962D932D1A08A02DAC
:100B300018199E2D98189E2D0301A02D1812181615
:100B40008616BA01BA0BA22D0800C7000C1EA62DEE
:100B5000470899008316981CAB2DAF2D8312831282
:100B6000080004304802C500831321308400C90105
:100B70000008C907840AC50BB82D0800831320306C
:100B800084005B308000840A4808E6203908800031
:100B9000840A38088000840A4A08E6203908800060
:100BA000840A38088000840A701DF32D083048023A
:100BB000C5000310C50C2530C60083171030F700A0
:100BC0008317770884000008E62083134608840012
:100BD00039088000C60A840A38088000C60A8317CC
:100BE000F70AC50BE02DB12503304802F60020308E
:100BF000760784004908E62039088000840A38080E
:100C00008000840A5D3080004808C50083132030CE
:100C1000840000086C25840AC50B092E0800831285
:100C200003138616831640309900831218121A088F
:100C30001A08181608008312031386168316153037
:100C40009900831218121A081A0818160800831639
:100C5000D0308700A00005148514851504309F004E
:100C6000831280309F000D278030CD00BA26080007
:100C700086157208CC0019278312031710308400E0
:100C80005726840A6326840A6F26840A7826840AF3
:100C90008526031383124C08F2007218E726F21817
:100CA000FA2672190D27F219192786110800031365
:100CB0008312AA2633301E02031C932E9A301E0282
:100CC0000318972E9B2E03138312AE265D081E0277
:100CD000031C932E5E081E020318972E9B2E0313EF
:100CE00083120D27A62624301E020318972E9B2E52
:100CF00003138312FA26AA2633301E02031C932EF6
:100D00009A301E020318972E9B2E03138312E72698
:100D1000A6260D275D081E02031C932E5E081E02E8
:100D20000318972E9B2E831701308000080083172D
:100D3000803080000800831700308000080083178F
:100D40001030840000308317800008009F121F12AB
:100D50009F11B22E9F121F129F15B22E9F121F16A7
:100D60009F15B22E55271F1455271F151F19B62E74
:100D70001F1008000313831286101130CB00C62603
:100D80004D08CB00C6268614592708000830BB0042
:100D9000CB0D031CCD2E8617CE2E8613000000002F
:100DA000000000000617000000000000000006130D
:100DB000BB0BC82E08008614061786170800861479
:100DC00006178613080086140617861308000708FE
:100DD000D1005115D1145110510887007214F2102E
:100DE0007211F2118A110A12D1208A110A120B1DF6
:100DF000F72E08000708D1005115D11051145108E1
:100E000087007210F2147211F2118A110A12D120A5
:100E10008A110A120B1D0A2F08000708D100511170
:100E2000D1145114510887007210F2107215F2118A
:100E300008000708D1005115D1145114510887003A
:100E40007210F2107211F215080094128316201617
:100E5000A0122008870083128516080094128316BA
:100E60002016A0162008870083128512080094120D
:100E70008316A0112008870083120515080094121C
:100E80008316A0152008870083120511080005129B
:100E900081010B110B1D4A2F7212080005168101EA
:100EA0000B110B1D512F72160800BA01BA0B562FE9
:100EB0000800CE200B1D5A2F0800FF30CF004F082E
:100EC000CD00BA26E726A6260D270530D0005F08FC
:100ED0001E02031C722FD00B672FCF0B5F2F003029
:060EE000CD00BA26080057
:100F20008207000010291C29552C242938294A2918
:100F30005C29682970297A298929A429552CBA297C
:100F4000BB29552CBC29C129552C552C552C552C69
:100F5000552C552C552C552CC729552C552CD4299E
:100F6000552C552C552C552CE129EE29FB29062A08
:100F7000112A1C2A272A322A422A822AA92AB22A7C
:100F8000C92AD02AD72AE32AEF2A0E2B212B552C47
:100F9000362B552C4E2B552C5F2B792B932B9B2BC3
:100FA000A92BB52BC12BCD2BD92BE52BF12BFD2B51
:100FB000092C172C232C2F2C3B2C452C4D2C552C3D
:040FC000552C0800A4
:101000000030E2000130E1001B27AA208A110A12F9
:1010100025278A150A1208001030E2000430E1008A
:101020001B270030E2007D08E2000F30E2057C085B
:10103000E1001B270030E2007A08E1001B27790855
:10104000E2007808E1001B27AA2008002030E20017
:101050000430E1001B277D08E2007C08E1001B272B
:101060000030E2007A08E1001B277908E2007808E6
:10107000E1001B27AA2008004030E2001330E10005
:101080001B270130E2007A08E1001B277908E20003
:101090007808E1001B2708005030E2003330E100FF
:1010A0001B270130E2007A08E1001B277908E200E3
:1010B0007808E1001B2708006030E2000430E100FE
:1010C0001B270030E2007A08E1001B277908E200C4
:1010D0007808E1001B2708007030E2000230E100D0
:1010E0001B270130E2007A08E1001B27AA20080034
:1010F000E2000330E1001B270130E2007A08E10042
:101100001B277908E2007808E1001B27AA200800C5
:10111000A030E2000330E1001B272F08E200300876
:10112000E1001B273108E2003208E1001B27AA205A
:101130008A110A1225278A150A120800B030E20027
:101140000130E1001B27AA208A110A1225278A15DF
:101150000A1208008A110A122E278A150A1202277B
:041160005327080009
:101200008A110A12CE208A150A120B1D0529080020
:101210007D08E3007C08E2000030E1003026203049
:10122000E3040030E1043D267908E3007808E20099
:101230000030E10030262030E3040030E1043D2698
:101240007E267E2608008A110A12372725278A154E
:101250000A12871287118A110A12E7268A150A12C2
:1012600008008A110A12372725278A150A128712C1
:1012700087118A110A12E7268A150A1208008A11B4
:101280000A120D278A150A128A110A12D1208A150C
:101290000A120B1D492908007E267E260430E30031
:1012A0000130E2000030E1003D267E267E26080067
:1012B00083160313250883120313E3008316031315
:1012C000240883120313E20030262030E3040030A8
:1012D000E1043D2683160313260883120313E3005B
:1012E00083160313230883120313E20030262030F1
:1012F000E3040130E1043D2683160313280883121A
:101300000313E30083160313270883120313E20079
:1013100030262030E3040230E1043D268316031317
:101320002B0883120313E300831603132A08831286
:101330000313E20030262030E3040330E1043D26AD
:10134000831603132C0883120313E300831603137D
:10135000290883120313E20030262030E30404300E
:10136000E1043D26831603132E0883120313E300C2
:10137000831603132D0883120313E2003026203056
:10138000E3040530E1043D26080083160313240816
:10139000F4002508F500831203137408E2007508B1
:1013A000E30030262030E3040030E1043D268316BC
:1013B00003132308F40083120313E3017408E2000B
:1013C00030262030E3040130E1043D260800750892
:1013D000E3007408E2000030E10030262030E3042E
:1013E0000030E1043D260800831603132508F500AC
:1013F0002408F400031383127508E3007408E20064
:1014000030262030E3040030E1043D268316031328
:101410002808F5002708F400031383127508E30079
:101420007408E20030262030E3040130E1043D2658
:10143000831603132B08F5002A08F4000313831204
:101440007508E3007408E20030262030E30402301F
:10145000E1043D26831603132E08F5002D08F40041
:10146000031383127508E3007408E200302620306D
:10147000E3040330E1043D260800EB30E3000330D1
:10148000E2000030E1003D267E267E267E267E2676
:10149000BB30E3000B30E200B630E1003D267E2693
:1014A0007E267E267E26BB30E300DB30E200B630AF
:1014B000E1003D267E267E267E267E26BB30E3008A
:1014C000EB30E200B630E1003D267E267E267E2609
:1014D0007E26BB30E3001B30E200B630E1003D2643
:1014E0007E267E267E267E26BB30E3000B30E20081
:1014F000B630E1003D267E267E267E267E26BB3047
:10150000E300DB30E200B630E1003D267E267E2699
:101510007E267E26BB30E300EB30E200B630E100F1
:101520003D267E267E267E267E26BB30E3001B30AF
:10153000E200B630E1003D267E267E267E267E260F
:101540000800EB30E3000330E2000030E1003D260C
:10155000BB30E3001B30E200B630E1003D267E26C2
:101560007E267E267E26BB30E3001B30E200B630AE
:10157000E1003D267E267E267E267E26BB30E300C9
:101580001B30E200B630E1003D267E267E267E2618
:101590007E26BB30E3001B30E200B630E1003D2682
:1015A0007E267E267E267E260800EB30E300033072
:1015B000E2000030E1003D26BB30E3001B30E200DA
:1015C0009630E1003D267E267E267E267E26080079
:1015D000EB30E3000330E2000030E1003D2608007C
:1015E000BB30E3001B30E2008630E1003D267E2662
:1015F0007E267E267E260800EB30E3000330E200E4
:101600000030E1003D26BB30E3000B30E200B63095
:10161000E1003D267E267E267E267E26BB30E30028
:10162000DB30E200B630E1003D267E267E267E26B7
:101630007E2608008830E3003C30E2002030E100E4
:101640003D260426831603132108A4002208A500C2
:10165000831203138830E3003C30E2002130E100C4
:101660003D260426831603132108A3002208A600A2
:10167000831203138830E3003C30E2002230E100A3
:101680003D260426831603132108A7002208A8007C
:10169000831203138830E3003C30E2002330E10082
:1016A0003D260426831603132108AA002208AB0056
:1016B000831203138830E3003C30E2002430E10061
:1016C0003D260426831603132108A9002208AC0036
:1016D000831203138830E3003C30E2002530E10040
:1016E0003D260426831603132108AD002208AE0010
:1016F0008312031308008830E3003C30E2002030FE
:10170000E1003D260426831603132108A4002208C5
:10171000A500831203138830E3003C30E20021303F
:10172000E1003D260426831603132108A7002208A2
:10173000A800831203138830E3003C30E20022301B
:10174000E1003D260426831603132108AA0022087F
:10175000AB00831203138830E3003C30E2002330F7
:10176000E1003D260426831603132108AD0022085C
:10177000AE00831203130800EB30E3000330E200F5
:101780008030E1003D26BA30E3000B30E200B63095
:10179000E1003D267E267E267E267E268830E300DA
:1017A0003C30E2002030E1003D2604260800EB300A
:1017B000E3000330E2008030E1003D26BA30E30070
:1017C0001B30E200B630E1003D267E267E267E26D6
:1017D0007E26BA30E3001B30E200B630E1003D2641
:1017E0007E267E267E267E26BA30E3001B30E2006F
:1017F000B630E1003D267E267E267E267E26BA3045
:10180000E3001B30E200B630E1003D267E267E2656
:101810007E267E260800EB30E3000330E2008030B5
:10182000E1003D26BA30E3001B30E2009630E100D3
:101830003D267E267E267E267E26BA30E300DB30DD
:10184000E200B630E1003D267E267E267E267E26FC
:10185000BA30E300DB30E200D630E1003D267E26E0
:101860007E267E267E26BA30E3001B30E200B630AC
:10187000E1003D267E267E267E267E26BA30E300C7
:101880001B30E2009630E1003D267E267E267E2635
:101890007E26BA30E300DB30E200B630E1003D26C0
:1018A0007E267E267E267E26BA30E300DB30E200EE
:1018B000D630E1003D267E267E267E267E26BA3064
:1018C000E3001B30E200B630E1003D267E267E2696
:1018D0007E267E260800EB30E3000330E200003075
:1018E000E1003D268830E3003B30E2001630E100A5
:1018F0003D268830E3003B30E2002630E1003D2603
:101900002030E3000430E2000730E1003D2608000B
:10191000EB30E3000330E2000030E1003D26883088
:10192000E3003B30E2001630E1003D262030E300CA
:101930000830E2000630E1003D268830E3003B300D
:10194000E2002630E1003D262030E3000430E200D2
:101950000730E1003D2608002030E3000030E200BF
:101960000630E1003D268830E3003B30E2001630CF
:10197000E1003D262030E3000730E200F630E100D0
:101980003D268830E3003B30E2002630E1003D2672
:101990002030E3000230E2000730E1003D2608007D
:1019A0002430E3000730E200FA30E1003D268830C1
:1019B000E3003B30E2000A30E1003D26080024301D
:1019C000E3000730E2005A30E1003D268830E300B2
:1019D0003B30E2000A30E1003D2608002430E300FD
:1019E0000730E2001A30E1003D268830E3003B304A
:1019F000E2000A30E1003D2608002430E300073011
:101A0000E2002A30E1003D268830E3003B30E2006E
:101A10000A30E1003D2608002430E3000030E200F7
:101A20001A30E1003D268830E3003B30E2000A3006
:101A3000E1003D2608002430E3000030E2000A30D7
:101A4000E1003D268830E3003B30E2000A30E1004F
:101A50003D2608002430E3000030E2008A30E10037
:101A60003D268830E3003B30E2000A30E1003D26AD
:101A700008002430E3000030E2004A30E1003D2657
:101A80008830E3003B30E2000A30E1003D260800E8
:101A90002430E3000030E2005A30E1003D26883077
:101AA000E3003B30E2000A30E1003D2608007E26DC
:101AB0007E260030E3007A08E2000030E1003026A4
:101AC0002030E3040030E1043D268830E30001309B
:101AD000E2009030E1003D267908E3007808E2005A
:101AE0000030E10030262030E3040630E1043D26DA
:101AF0007E267E2608000030E3007A08E2000030EF
:101B0000E10030262030E3040030E1043D26883037
:101B1000E3000130E2009030E1003D267908E30067
:101B20007808E2000030E10030262030E30407307E
:101B3000E1043D2608002030E3000530E200583083
:101B4000E1003D262030E3000A30E200A930E10048
:101B50003D268830E3003B30E2003830E1003D268E
:101B60008830E3003B30E2003930E1003D260800D8
:101B70002030E3000430E2000730E1003D2643302E
:101B8000E3000330E2000730E1003D26AF30E30020
:101B90000030E2004230E1003D26EC30E300273027
:101BA000E2006430E1003D268830E3003B30E20093
:101BB0001630E1003D2608004330E3000330E20028
:101BC0000730E1003D268830E3003B30E20016306C
:101BD000E1003D260800A830E300E730E200613074
:101BE000E1003D267E267E267E267E2600210021DF
:101BF000A930E300E730E2006130E1003D267E26B7
:101C00007E267E267E2608008A110A1225278A153E
:101C10000A127E264A260830BB0087158711BB0BA7
:101C20000D2E8A110A122E278A150A121030BB00B7
:101C300087150310071A03148711F50CF40CBB0B5E
:101C4000182E7E268A110A1225278A150A12831653
:101C500003137508A2007408A1008312031308007F
:101C60000430BB000310E30CE20CE10CBB0B322E82
:101C70000F30E305F030E105080087128715871162
:101C80008712871587118712871587118712871585
:101C90008711572E87168715871187128715871189
:101CA000871287158711871287158711080008305A
:101CB000BB00E10C87120318871687158711BB0B31
:101CC000592EE10C871200000830BB00E20C87128D
:101CD0000318871687158711BB0B662EE20C871237
:101CE00000000830BB00E30C871203188716871525
:101CF0008711BB0B732EE30C87120800E301E2018E
:101D0000E1013D2608007B08E3007A08E200E101DA
:101D100030262030E3040630E1043D268830E3001D
:101D20003B30E2002630E1003D267908E3007808E8
:101D3000E200E10130262030E3040630E1043D26D4
:101D40008830E3003B30E2001630E1003D26080019
:101D5000BA30E3000230E2009630E1003D267E26F4
:101D60007E267E267E260800BB30E3001B30E20084
:101D70008530E1003D267E267E267E267E260800D2
:101D8000A030E300B030E2000530E1003D2608005D
:101D9000A130E300B030E2000530E1003D2608004C
:101DA000A030E300F030E2000530E1003D260800FD
:101DB000A130E300F030E2000530E1003D260800EC
:101DC0008A110A12372725278A150A1287168715BE
:101DD0008A110A16EC258A150A12871287118A11B0
:101DE0000A12CB208A150A120B1DF42EFF30E400D4
:101DF0000000E40BF82E08008A110A120D278A153C
:101E00000A120800FC3081000B11071A0A2F0B1D63
:101E1000052F192F7F3081000B11071E122F0B1D6C
:101E20000D2F192FFF3081000B110B1D152F0030C6
:101E30001A2FFF3008008A110A1225278A150A1264
:101E40000830BB00E20D87120318871687150000C3
:101E50008711BB0B222FE20D871200000830BB0058
:101E6000E10D871203188716871500008711BB0B39
:101E7000302FE10D871200000330E4000000E40B76
:101E80003E2F08001030BB0087150310071A0314FB
:101E90008711F40DF50DBB0B442F0830E400000052
:101EA000E40B4F2F080042271330E4000000E40B3E
:101EB000562F831203137408E5007508E6004227C5
:101EC000831203137408E7007508E800E61A692F07
:0A1ED0006A2F000008000800080057
:102000008A150A1223214C2108213F218A110A1620
:1020100008008A110A12AA268A110A1676301E02B0
:10202000031C7A2813288A150A1223218A110A16FA
:102030008A150A124C218A110A16F830FA0000306B
:10204000F9000630F8008A150A125725BC238A11B8
:102050000A1683160313220883120313F600313085
:1020600076060319662883160313220883120313C6
:10207000F60033307606031966283E288A150A12C0
:102080002A258A110A160230D800F830FA000030EA
:10209000F9000630F8008A150A127B258A110A1603
:1020A0008A150A12E8228A110A168A150A12F022E3
:1020B0008A110A168A150A129B258A110A168A1590
:1020C0000A12EB258A110A16D80B4528831203132E
:1020D0000030FB008030FA000030F9008030F8005A
:1020E0008A150A128326D0249B25EB253F218A11CD
:1020F0000A1608000230D8008A150A122A257B2504
:10210000E822F0229B25EB258A110A16D80B7C28A1
:102110000130FE008030FD000030FC00F801F901C4
:10212000FA01FB014030DB002123003A0319B828F3
:102130008A150A1231214C2183268A110A16403051
:10214000F807031CAF280130F907031CAF28013042
:10215000FA07031CAF280130FB07031CAF288A15C0
:102160000A12EE249B25EB253F218A110A1694289A
:10217000F1207F30FA00F030F9000030F800FF0164
:10218000FE010F30FD00FF30FC000F30DB0021238B
:10219000003A0319EB288A150A1223214C218326C1
:1021A0008A110A162030F807031CE2280130F907CB
:1021B000031CE2280130FA07031CE2280130FB0768
:1021C000031CE2288A150A12DF249B25EB253F21F8
:1021D0008A110A16C7288A150A123F218A110A167F
:1021E00008008030FA000030F9000030F800FF01EC
:1021F000FE010630FD000030FC004030DB002123F2
:10220000003A031923298A150A1231214C21832609
:102210008A110A164030F807031C1A290130F90701
:10222000031C1A290130FA07031C1A290130FB0785
:10223000031C1A298A150A12EE249B25EB253F213F
:102240008A110A16FF28080008008A110A12AA2615
:102250008A110A1676301E02031CB9282F298A1506
:102260000A1223214C219B25EB253F218A110A16B6
:1022700008008A150A1223214C219B25EB253F21BA
:102280008A110A1608008A110A12AA268A110A1649
:1022900076301E02031CF1284D298A150A122321CB
:1022A0004C218A110A16F1208A150A123F218A113F
:1022B0000A16080083171030840001308000840A59
:1022C00003308000840A0230800008008317103039
:1022D00084000A3080000800F1120130DB008A150A
:1022E0000A1223214C212A257B258A110A16212333
:1022F000003A031996298A150A122A257B258A1184
:102300000A168A110A123925F4003925F5008A11B6
:102310000A168A150A12E721D5229B25EB258A1178
:102320000A160230F8070318F90A77298A150A12E3
:102330003F218A110A160800C1080319AC298A1521
:102340000A12E02600208A110A1663258A150A124D
:10235000FC268A110A160800F1128A150A12232196
:102360004C2148257B258A110A16DA013C2359089D
:10237000003A0319DE298A150A1248257B258A119D
:102380000A161030DA000430D8000E248A150A121A
:10239000F421A1228A110A16DA03DA03DA03DA0336
:1023A000D80BC5298A150A129B25EB254C218A11C9
:1023B0000A162030F8070318F90AB729DA080319B2
:1023C000002A83160313FF30A500A400A800A7006D
:1023D000AB00AA00AE00AD00031383128A150A12E7
:1023E000F421A1228A110A16DA03DA03DA03DA03E6
:1023F000031DDE298A150A129B25EB258A110A1670
:102400008A150A123F218A110A160800F1120430B7
:10241000DB008A150A1223214C218A110A168A151B
:102420000A124C218A110A162123003A0319192A8B
:102430000F2A8A150A123F218A110A160800C108BC
:1024400003192F2A8A150A12E02600208A110A167B
:102450009F258A150A12FC268A110A160800F11215
:102460008A150A1223214C210C257B258A110A1674
:10247000DA013C232030DA000830D8005908003A4D
:102480000319612A8A150A120C257B258A110A165E
:102490005F248A150A1258213D228A110A16DA038E
:1024A000DA03DA03DA030830F8070318F90AD80B5D
:1024B0003E2A8A150A129B25EB254C218A110A1601
:1024C0003A2ADA080319872A83160313FF30A30078
:1024D000A500A400A600A800A700A900AB00AA00C0
:1024E000AC00AE00AD00031383128A150A12582106
:1024F0003D228A110A16DA03DA03DA03DA03031D2E
:10250000612A8A150A129B25EB258A110A168A155B
:102510000A123F218A110A160800F1128A150A12BE
:1025200023214C218A110A163C238A150A124C21B8
:102530008A110A165908003A0319A82A8A150A129C
:102540005725BC238A110A16C024F80AF80A952ACE
:102550008A150A123F218A110A160800C1080319B8
:10256000BE2A8A150A12E02600208A110A1645257D
:102570008A150A12FC268A110A160800F1128A1519
:102580000A1223214C2157258A110A163C23590887
:10259000003A0319DC2A8A150A12D7237B238A11F1
:1025A0000A16BD238A150A124C218A110A16043014
:1025B000F8070318F90AC72A8A150A123F218A1157
:1025C0000A160800C1080319F22A8A150A12E02621
:1025D00000208A110A16E6248A150A12FC268A119E
:1025E0000A160800F1128A150A1223214C215725D8
:1025F0008A110A163C235908003A0319192B8A1527
:102600000A1257250B241A238A110A165C238A15ED
:102610000A124C218A110A160830F807031C182BDD
:102620000130F907031C182B0130FA07031C182B83
:10263000FB2A8A150A123F218A110A1608002F2246
:1026400008008A110A16FF08031D2F2BFE08031D20
:102650002F2BFD08031D2F2BFC08031900345B08EA
:10266000FC0203183B2B0130FD0203183B2BFE023A
:1026700003183B2BFF02FF348A110A16FF08031DC3
:102680004D2BFE08031D4D2BFD08031D4D2BFC0893
:10269000031D4D2B0030D90008000130FC02031847
:1026A000592B0130FD020318592BFE020318592B38
:1026B000FF02FF30D9000800831603132408F4003A
:1026C0002508F5002308F300831203138A110A1268
:1026D0007408312575083125730831258A110A16C9
:1026E0003C235908003A0319BC2B8316031327080F
:1026F000F4002808F5002608F300831203138A115A
:102700000A127408312575083125730831258A119C
:102710000A163C235908003A0319BC2B83160313ED
:102720002A08F4002B08F5002908F300831203138C
:102730008A110A127408312575083125730831256C
:102740008A110A163C235908003A0319BC2B831638
:1027500003132D08F4002E08F5002C08F300831253
:1027600003138A110A12740831257508312573087C
:1027700031258A110A163C23080083160313250805
:10278000F5002408F400831203138A110A12740856
:102790003125750831258A110A163C235908003A5B
:1027A00003190D2C831603132808F5002708F400DD
:1027B000831203138A110A12740831257508312512
:1027C0008A110A163C235908003A03190D2C831666
:1027D00003132B08F5002A08F400831203138A114F
:1027E0000A1274083125750831258A110A163C230E
:1027F0005908003A03190D2C831603132E08F5000F
:102800002D08F400831203138A110A12740831256B
:10281000750831258A110A163C2308008A110A120C
:102820003925F4003925F5008A110A168316031399
:102830007408A4007508A500831203133C235908EB
:10284000003A03195E2C8A110A123925F400392541
:10285000F5008A110A16831603137408A700750879
:10286000A800831203133C235908003A03195E2C75
:102870008A110A123925F4003925F5008A110A1641
:10288000831603137408AA007508AB0083120313A0
:102890003C235908003A03195E2C8A110A12392583
:1028A000F4003925F5008A110A16831603137408FB
:1028B000AD007508AE00831203133C2308008A1193
:1028C0000A123925F4003925F5003925F3008A115B
:1028D0000A16831603137408A4007508A50073086C
:1028E000A300831203133C235908003A0319BF2C99
:1028F0008A110A123925F4003925F5003925F3002B
:102900008A110A16831603137408A7007508A80015
:102910007308A600831203133C235908003A0319D5
:10292000BF2C8A110A123925F4003925F500392502
:10293000F3008A110A16831603137408AA00750897
:10294000AB007308A900831203133C235908003A13
:102950000319BF2C8A110A123925F4003925F50014
:102960003925F3008A110A16831603137408AD0083
:102970007508AE007308AC00831203133C230800F3
:10298000831603132108F4002208F50083120313B1
:1029900074088A110A1231258A110A1675088A11DB
:1029A0000A1231258A110A163C2308000334033425
:1029B00002340234023402340130DC0008000230F8
:1029C000DC0008000230DC00080000348A150A121E
:1029D00026208A110A163C235908003A0319F32CC1
:1029E000F4241C25EC2C08008A150A1242278A11AF
:1029F0000A16831603137408A4007508A500831231
:102A000003138A150A1242278A110A168316031322
:102A10007408A3007508A600831203138A150A120E
:102A200042278A110A16831603137408A700750833
:102A3000A800831203130800831603138A110A12D5
:102A400024088312312583160313250883123125A8
:102A5000831603132308831231258A110A163C2397
:102A6000831603138A110A1227088312312583164D
:102A700003132808831231258316031326088312B3
:102A800031258A110A163C2308008A150A120C20E7
:102A90008A110A163C235908003A0319572D8A1542
:102AA0000A1242278A110A1658253C234B2D08008A
:102AB000831203138A110A1274083125750831250F
:102AC0008A110A1608001030DB002123003A03198E
:102AD0007E2D2030D8007F2580308A150A1278207C
:102AE0003C208A110A168C258A150A12AA208A11FE
:102AF0000A162030F8070318F90A652D0800831715
:102B0000103084008A110A1239258A110A168000B1
:102B1000840AD80B822D08008317103084001030EF
:102B2000D8000008E100840A0008E200840A8A153F
:102B30000A121B278A110A16D80B912D0800203083
:102B4000DB002123003A0319BC2D6030D8007F251B
:102B500090308A150A1278204C208A110A16BD2559
:102B60008A150A12AA208A110A164030F80703189B
:102B7000F90A0319FA0AA12D0800831710308400FE
:102B80001030D800C625D80BC22D08000008E1007F
:102B9000840A0008E2008A150A121B278A110A1605
:102BA000840A0008E100840A840A840A0008E2001A
:102BB0008A150A121B278A110A1684038403000847
:102BC000E100840A0008E2008A150A121B278A1114
:102BD0000A16840A840A0800031383120708D10026
:102BE0005115D1145110510887007214F21072114E
:102BF000F2118A110A12CB208A110A160B1DFE2D22
:102C000008007130DD00A230DF00A930DE008A113B
:0C2C10000A125D278A110A16080008004D
:103000000800031383160030940083129412080002
:10301000831203130130550603195B28023055064D
:10302000031967280330550603196E280430550626
:1030300003198028053055060319922806305506D5
:1030400003199E28073055060319AA28083055068B
:103050000319B628093055060319C2280A30550647
:103060000319D4280B3055060319E6280C305506F1
:103070000319EC280D30550603192A290E30550680
:10308000031964291830550603197129193055069A
:1030900003197E291A305506031980291B3055065D
:1030A000031982291C305506031983291D30550642
:1030B000031995290800A721711866281A22831779
:1030C0001030840056088000831203130800A721E3
:1030D00071186D280330D200E4210800A72171186F
:1030E0007F288A110A16D824D2008A150A16EE21E2
:1030F0008A110A16D924D2008A150A160422080059
:10310000A721711891288A110A16D824D2008A158D
:103110000A16EE218A110A16D924D2008A150A1637
:1031200004220800A72171189D288A150A16D200CA
:10313000EE218A150A16D20004220800A721711870
:10314000A9288A150A16D200EE218A150A16D2007D
:1031500004220800A7217118B5288A150A16D20082
:10316000EE218A150A16D20004220800A721711840
:10317000C1288A150A16D200EE218A150A16D20035
:1031800004220800A7217118D3288A110A16D62410
:10319000D2008A150A16EE218A110A16D724D20007
:1031A0008A150A1604220800A7217118E5288A1139
:1031B0000A16D624D2008A150A16EE218A110A169A
:1031C000D724D2008A150A1604220800A721D701A5
:1031D000721BD70A36220800F110831203137C08F1
:1031E000D7003622F119F1147D08D7003622F119E3
:1031F000F1147E08D7003622F119F1147808D700AF
:103200003622F119F1147908D7003622F119F11498
:103210007A08D7003622F119F11417298A110A12F7
:1032200039258A150A16D7003622F119F114FE083D
:10323000031D2029FD08031D2029FC080319292945
:103240000130FC0203180E29FD0203180E29FE02AC
:103250000E290800A721711863298A110A16D7249C
:10326000D2008A150A168317103084008001840A60
:103270008001840A8001840A8001E42183171030D0
:103280008400840A840A840A0008D4001030840070
:103290000008840A840A840A8000103084005408DC
:1032A0008000831710308400840A840A0008D40048
:1032B00010308400840A0008840A800010308400E2
:1032C000840A540880000800A72171187029780822
:1032D000D70036227908D70036227A08D70036225E
:1032E0000800A72171187D297808D70036227C08AC
:1032F000D70036227D08D70036220800A721080013
:10330000A72108000800A7217118D3288A110A16DE
:10331000DA24D2008A150A16EE218A110A16DB2455
:10332000D2008A150A1604220800A7217118E52880
:103330008A110A16DA24D2008A150A16EE218A1199
:103340000A16DB24D2008A150A160422080071101E
:103350005508D7003622FF30D6001A2256085702E9
:10336000031D7114D608031DB72971141A22080011
:103370008A110A1621238A150A16003A0319CE2942
:103380005C08D2001A22711ACE2956088A110A1234
:1033900031258A150A16D20BC229B82908008A11CC
:1033A0000A1621238A150A16003A0319E3295C0834
:1033B000D2008A110A1239258A150A16D700362238
:1033C000D20BD929CF2908008317103084001A2284
:1033D00056088000840AD20BE72908007808D70035
:1033E0003622D2030319032A7908D7003622D203E2
:1033F0000319032A7A08D7003622D2030319032AB5
:103400007B08D700362208007C08D7003622D2037A
:103410000319192A7D08D7003622D2030319192A65
:103420007E08D7003622D2030319192A7F08D70055
:103430003622080093015122F1192D2A71128A11A6
:103440000A122E278A150A162530940094168C111C
:103450008C1D282A1308D6002E2A711687128A116D
:103460000A12252794128A150A1608005122F1190A
:10347000422A2530940094168C11570893008C1D15
:103480003F2A422A8A110A12CB208A150A160B1DDE
:10349000472A87128A110A12252794128A150A16BA
:1034A00008008A110A123F2725278A150A16F111EA
:1034B0008A110A12D1208A150A160B196E2A871D45
:1034C0005D2A78228716F1118A110A12D1208A15F5
:1034D0000A160B196E2A8719692A6F2AF115080036
:1034E000080008008A110A12C8208A150A16892ABB
:1034F0008A110A12CB208A150A16892A8A110A1201
:10350000CE208A150A16892A8A110A12D1208A1514
:083510000A160B1D892A0800B0
:043518000034003447
:00000001FF
